:060000000A128A11122809
:10000800FE00030EF6000408F7000A08F800831241
:1000180003137F08F9000A128A11C02A0A128A11EA
:10002800152883120313CB0183010A128A111C2895
:100038007030831603138F04831603178801890110
:100048008312031385018601870183160313850133
:100058000330860010308700831203170508E13942
:100068001638850083160313811583120313940130
:100078008316031314178312031394160A128A1192
:10008800B2260A128A111A3083120313BF00F730FE
:10009800BE00BE0B4D28BF0B4D28522800300A1257
:1000A8008A111E210A128A110A128A11DA240A12E6
:1000B8008A11CC300A128A11FE250A128A1144309C
:1000C8000A128A11FE250A128A110A3083120313B2
:1000D800C0002230BF00A030BE00BE0B7128BF0B8D
:1000E8007128C00B712800000A128A11DA240A123A
:1000F8008A11CC300A128A11FE250A128A11BE30E2
:100108000A128A11FE250A128A110A128A11A525D5
:100118000A128A1183120313BE003E08C5000A1290
:100128008A11A5250A128A1183120313BE003E08FC
:10013800C6000030AE008030AF004130B000450846
:10014800BE00BF014608C000C1014008C100C0018F
:100158003E084004A8003F084104A9000A128A1179
:100168005D250A128A11831203132808B100290891
:10017800B2002A08B3000A128A1108220A128A1148
:10018800831203132E08C7002F08C8003008C900BF
:100198004730BE003E08CA004A088400831300089E
:1001A800BE003E08C4000130BE003E08CA074A0827
:1001B80084000008BE003E08C3000130BE003E08AF
:1001C800CA074A0884000008BE003E08C20003307F
:1001D800BE003E08A50042300A128A1148240A12BD
:1001E8008A11823083120313BF00DD30BE00BE0BBC
:1001F800FB28BF0BFB288312031705140630831254
:100208000313BF002F30BE00BE0B0829BF0B0829FF
:100218000D296300000000008312031705100D303C
:1002280083120313BF00FB30BE00BE0B1929BF0B9E
:100238001929582883120313AC000230AB002B088D
:10024800A30005300A128A1116260A128A110730ED
:1002580083120313AB002B08A30006300A128A117D
:1002680016260A128A11083083120313AB002B08D2
:10027800A30000300A128A1116260A128A111F30AA
:1002880083120313AB002B08A30004300A128A114F
:1002980016260A128A11E629E73083120313B100E1
:1002A800B000AF00AE00AB002B08AD002D300A1235
:1002B8008A117E260A128A112D300A128A115626B0
:1002C8000A128A11FC29C23083120313B100B0004C
:1002D800AF00AE00AB002B08AD002D300A128A111A
:1002E8007E260A128A112D300A128A1156260A12FF
:1002F8008A11FC29C23083120313B100B000AF0089
:10030800AB002B08AE00C330AB002B08AD002D307E
:100318000A128A117E260A128A112D300A128A11AF
:1003280056260A128A11FC29C23083120313B1001F
:10033800B000AF00AB002B08AE00C430AB002B08F8
:10034800AD002D300A128A117E260A128A112D302C
:100358000A128A1156260A128A11FC29C2308312FF
:100368000313B100B000AF00AB002B08AE00C530DE
:10037800AB002B08AD002D300A128A117E260A1216
:100388008A112D300A128A1156260A128A11FC295E
:10039800C23083120313B100B000AF00AB002B08CA
:1003A800AE00C630AB002B08AD002D300A128A1102
:1003B8007E260A128A112D300A128A1156260A122E
:1003C8008A11FC29831203132C08003A03195029B7
:1003D800013A03196729033A03197E29013A0319D7
:1003E8009829073A0319B229013A0319CC29FC299B
:1003F80083120313CB010A30AB002B08A300003093
:100408000A128A1116260800831203133108B40051
:100418003208B5003308B6000310350D360DB700A5
:100428003708BC003C08031D202A0030AE0000300D
:10043800AF000030B00008002E08B4002F08B50047
:100448003008B6000310350D360DB7003708BD006B
:100458003D08031D362A0030AE000030AF000030E2
:10046800B00008000030B9000030BA000030BB000E
:1004780089303D07B4003408BC023108B4003208A2
:10048800B5003308B60010300310B60CB50CB40C28
:10049800FF3E031D482A3408B7003708BD002E0860
:1004A800B4002F08B5003008B60010300310B60CA1
:1004B800B50CB40CFF3E031D5A2A3408B7003708A0
:1004C800BD068030B4003408BD05B217FF30B10551
:1004D800FF30B2050030B305AF17FF30AE05FF306F
:1004E800AF050030B0051830B4003408B80001304A
:1004F8000310B90DBA0DBB0DFF3E031D7C2A300851
:100508003302031D8D2A2F083202031D8D2A2E085F
:100518003102031C9A2A2E08B1022F08031C2F0F40
:10052800B2023008031C300AB30239140130031038
:10053800B10DB20DB30DFF3E031D9B2A0130B80269
:10054800031D7B2A3908A0003A08A1003B08A20035
:100558003C08B4003408A3003D08B5003508A400E1
:100568000A128A11DA23831203132008AE00210825
:10057800AF002208B000080077300A128A118225DD
:100588000A128A118B1C4E2B8B1083120313051031
:10059800FF300A128A1141260A128A11F5007508DD
:1005A800FB008312031305147B09F5007508FA0094
:1005B80000007B1FF12A2D300A128A1182250A12A7
:1005C8008A11831203130510E2300A128A11412698
:1005D8000A128A1183120313051400007B1E1C2BB8
:1005E80001300A128A1182250A128A118312031312
:1005F8000510E1300A128A1141260A128A11831263
:10060800031305141030F5007508F30007300A12BB
:100618008A116A260A128A11831203138517093070
:10062800F500F50B152B182B831203138513CB013B
:10063800FB1E3A2B4B300A128A1182250A128A11A4
:100648002030F5007508F30007300A128A116A266F
:100658000A128A118312031385170930F500F50B66
:10066800332B362B831203138513CB017B1C4E2BA4
:1006780068300A128A1182250A128A11831203131A
:100688000510E1300A128A1141260A128A118312D2
:1006980003130514790883120313FF0078088A00EE
:1006A80077088400760E8300FE0E7E0E0900033064
:1006B8008A000408840A820700344D34613478348F
:1006C80069346D3475346D3420346E3475346D345A
:1006D80062346534723420346F34663420345434D0
:1006E80058342034723465347434723461346E345E
:1006F80073346D34693474347334203469346E342B
:1007080074346534723472347534703474340A3421
:1007180000344434613474346134203452346534E0
:1007280061346434793420345234583420344634B3
:10073800493446344F34203469346E347434653463
:10074800723472347534703474340A340034443476
:100758006134743461342034533465346E34743401
:1007680020345434583420344634493446344F34D1
:10077800203469346E3474346534723472347534A8
:10078800703474340A340034543458345F34463482
:1007980055344C344C340A34003431340A3400347F
:1007A80032340A34003435340A34003483120313E3
:1007B80023080319E42B220821042004031DF72B26
:1007C8000030A0000030A1000030A2000800013075
:1007D800A5002508A30701300310A20CA10CA00C4A
:1007E800FF3E031DF02BFE3022050319122CEB2BC4
:1007F8000130A5002508A3070130A0070030031821
:100808000130A107003003180130A207013003109E
:10081800A20CA10CA00CFF3E031D0B2CFF302205DF
:100828000319212CFC2B0130A30201300310A00D69
:10083800A10DA20DFF3E031D1A2CA11B272C02306F
:1008480023020318172C23182F2CFF30A0057F3004
:10085800A105FF30A2050310A30C2308A500A601DB
:10086800A70110300310A50DA60DA70DFF3E031D0F
:10087800362C2508A0042608A1042708A204240869
:1008880003190800A217080083120313A700713088
:100898000A128A1134250A128A11000083120313DE
:1008A8004B08031D522C74300A128A1134250A127F
:1008B8008A1100008312031385130130A60026084D
:1008C800CB000A30A6002608A30000300A128A11BD
:1008D80016260A128A11633083120313A600A60B88
:1008E800732C0000831203130510E1300A128A11D9
:1008F8008E260A128A118312031305140510A030DC
:100908000A128A118E260A128A11831203132508E5
:10091800A6002608A00027080A128A11C6250A126E
:100928008A118312031305148517053083120313E4
:10093800A600A60B9D2CA02C831203138513080078
:1009480083120313A10021080319C22C0A128A1169
:10095800C9260A128A11033083120313A000A00BC0
:10096800B32C0A128A11D0260A128A11293083124E
:100978000313A000A00BBE2CC12C08000A128A1178
:10098800C9260A128A11273083120313A000A00B6C
:10099800CB2C0A128A11D0260A128A11053083122A
:1009A8000313A000A00BD62CD92C08000A128A1118
:1009B800C9260A128A11BF3083120313A100E42C3E
:1009C800A10BE32CE72C0A128A11D0260A128A11ED
:1009D8002D3083120313A100A10BF02CF32C0A1263
:1009E8008A119E260A128A1183120313A100210874
:1009F800A200A33083120313A100022DA10B012D25
:100A0800052D0A128A11D02608000A128A11C92651
:100A18000A128A11033083120313A100A10B122DAD
:100A28000A128A11D0260A128A110530831203137A
:100A3800A100A10B1D2D0A128A119E260A128A11E5
:100A480083120313A1002108A20023308312031389
:100A5800A100A10B2D2D302D8312031322080800AD
:100A680083120313A1000A128A11AA260A128A11F4
:100A7800003A031D372D83120313210884000A123C
:100A88008A115B230A128A110A128A11D7260A12BE
:100A98008A11013083120313A107FF302107840054
:100AA8000A128A115B230A128A11003A03190800F4
:100AB800372D83120313AD01A91F692DA809A909B0
:100AC800A80A0319A90AAD01AD0A2808A000290837
:100AD800A100A2018E30AB002B08A3002D08AC00AA
:100AE8002C08A4000A128A11DA238312031320089F
:100AF800A8002108A9002208AA000800F1000A128B
:100B08008A11BA260A128A11003A031D832D710828
:100B180084000A128A115B230A128A110A128A11A6
:100B2800DD260A128A110130F107FF3071078400AF
:100B38000A128A115B230A128A11003A0319080063
:100B4800832D83120313A401A5010830250203187D
:100B5800C42D0310A40C0A128A1109250A128A113D
:100B6800003A0319BA2D83120313A4170130831214
:100B78000313A3002308A50708302502031CAE2D84
:100B88002408080083120313A200A30120082302EB
:100B98000318080023082207A100210884008313F2
:100BA8000008930083160313141CD62D8312031315
:100BB8008C1DD62D8C110130A1002108A307CA2D48
:100BC80083120313A700051027081F3920380A12BB
:100BD8008A112C260A128A11831203132508A600EB
:100BE8002608A00024080A128A11C62583120313B6
:100BF8000514080083120313A300A401083024027B
:100C080003180800230801390A128A11A4240A12B9
:100C18008A11031083120313A30C0130A2002208C7
:100C2800A407022E83120313A400051024081F39F9
:100C380020380A128A112C260A128A1183120313E9
:100C480023080A128A112C2683120313051408009C
:100C580083120313A100A201210893008316031332
:100C6800141C322E831203138C1D322E8C11130880
:100C7800A0002008A20022080800F100F201710873
:100C880083120313930083160313141C472E831235
:100C980003138C1D472E8C111308F0007008F20006
:100CA8007208080083120313AA0085132A08A800F3
:100CB8002808A4000530A9002908A5000A300A124E
:100CC8008A11E4258312031385170800F4008312A0
:100CD8000313051074081F3920380A128A11412697
:100CE8000A128A1173080A128A1141268312031301
:100CF8000514080083120313AA002A08A80028086C
:100D0800A4000530A9002908A50010300A128A118C
:100D1800E425080083120313A2001308A00020088A
:100D2800A1008C11941322089300941B08008C19BD
:100D380008009B2E83120313A0018614861CA72E7D
:100D4800A001A00AA82EA0012008080083160313FA
:100D58009818B02E013008000030080083120313E1
:100D6800851305140A128A11C22608008316031374
:100D78009818C02E013008000030080083160313AD
:100D880001130B168B108B1708008316031386109C
:100D98008312031386100800831603138610831228
:100DA80003138614080083120313A0002008990077
:0E0DB8000800F0007008831203139900080071
:04400E00D4ECFFFFF0
:00000001FF
